:020000040000FA
:040000006028423002
:08000800A000030EA100831209
:1000100005191028831601178312B2308100542865
:1000200083160113831203140B190310A80D2E1B42
:100030002E28A50DA516FF302502031D5428FB30E0
:100040002802031D26284E30AE005428FC3028021A
:10005000031D54284630AE00A70154280318542825
:10006000AE1D39282808A700AE11270A03194E280B
:1000700052282E1D3F282808A6002E115228AE1CFB
:1000800045282808A500AE1052282D152708AB00DA
:100090002608AA002508A9002808AC00AE01A8017E
:1000A000A5015428FF30A8008B100B11210E8300EE
:0600B000A00E200E090065
:1000C000203084008001840A80300402031C6228EE
:1000D000C5218501870183160C30850587018312B0
:1000E00083160514871507168312850187010730CB
:1000F000990000309A00103083168E008312603011
:1001000083168F0083120030831691009F008312A4
:10011000C83083168100831231309000003083167E
:100120008C00831210308B00831600309B001C144F
:100130001A088312BD00851D0027831610309B000E
:100140001C141A088312BE00092281018E018F013E
:100150000B118B100B108C018B17BC202D19BE209E
:10016000B30BBA28031085190314BA0DF0303A0204
:1001700003192921C023AD2864000800A91F080025
:10018000291B08002B082A0629062C02031D08003B
:100190002D110130B7008B132030370783169B00D9
:1001A0001C141A088312A4001030370783169B0012
:1001B0001C141A088312A3000030370783169B0013
:1001C0001C141A088312A2008B1724082B02031D8B
:1001D000232923082A02031D2329A91E29122208E4
:1001E0002906F039031D2329220829050F3903198F
:1001F0000B2901303702031D02293E1802293E1443
:100200003F14F92102303702031D0B29BE180B29B8
:10021000BE143F14FD21290922050F390319232992
:1002200001303702031D19293E1C19293E103F14C5
:10023000012202303702031D2229BE1C2229BE10D2
:100240003F1405222329B70A033037020318080098
:10025000CB283D1C0800B601B3019630B400013034
:10026000B5000130B70085018701AD138F21BC2097
:10027000B30B5029031085190314BA0DF0303A025C
:1002800003197F29B41F0710B40B50293708B6088B
:100290000319B60003194E290714B6039630B400AB
:1002A0002D1D37292D11A91F3729291B3729A91ED3
:1002B00029120F30290503193729B9012918B90A5C
:1002C000A918B90A2919B90AA919B90AB9183729EF
:1002D000391937298B1320303707BC002B08BB0096
:1002E000B02110303707BC002A08BB00B021003015
:1002F0003707BC002908BB00B0218B178921850175
:100300008701B70AB60103303702031C37290922D7
:1003100008000230370203190800850187011430F4
:10032000B90001300F1E87000F1A8701BC202D1D58
:1003300091292D11A91F9129291B91290F302905D8
:10034000031D8F29B90B91298501870108003F1CE6
:1003500008003F101030BC003E08BB00B021080070
:100360008B133B0883161C159A0083123C088316D6
:100370009B0055309D00AA309D009C1464009C1881
:10038000BE291C1183128B170800003095006030C5
:1003900084008B13831604089B001C141A08831214
:1003A0008B178000840A68300402031CC92964305A
:1003B000D5002D24DC003C30EC00ED00EE00EF0019
:1003C000EA146E30D5002D240F39031D08003224A5
:1003D0000F39031D080037240F39031D08003C2482
:1003E0000F39031D08008316871107128312EA10C4
:1003F00008000130E800182208000430E800182244
:1004000008000230E800182208000830E80018222E
:100410000800EA178B13831670309B001C141A080F
:1004200083128B17E80018220430EB00EA1308004F
:10043000E80803190800681C252A6730D5002D2418
:10044000D1006830D5002D24D200E81C2F2A673057
:10045000D5003224D1006830D5003224D200681D86
:10046000392A6730D5003724D1006830D5003724C9
:10047000D200E81D432A6730D5003C24D100683003
:10048000D5003C24D200681E4D2A6A30D5002D24A8
:10049000D1006B30D5002D24D200E81E572A6A30D7
:1004A000D5003224D1006B30D5003224D200681F31
:1004B000612A6A30D5003724D1006B30D50037244B
:1004C000D200E81F6B2A6A30D5003C24D1006B3083
:1004D000D5003C24D200EA16D11A7B2A511B7B2A74
:1004E000511C7B2ADC1FEA125C1F7B2A501C7B2AD2
:1004F000C01B7B2A0800EA1E8B2AEA1B8B2A511894
:1005000070308B1383169B001C141A0883128B17F0
:10051000680203190800D11A962A511B962A6A10FC
:10052000511C962A5014051E6A140516511C9E2A49
:10053000511A5016D11AC017511B5012EA1FA52A82
:10054000D11A0800511B0800A92AD11AD62A511B1A
:10055000D62A6530D500521A2D24D21A3224521BC5
:100560003724D21B3C245118C4006630D500521ADF
:100570002D24D21A3224521B3724D21B3C2451186A
:10058000CC0052085118D70004306A183230EA1BE8
:1005900032305118C80051185C14EA1FD42A511C7B
:1005A000D32A4403C00008005118C001511870300C
:1005B000BC006808E900BB00B021BE010800FD01D5
:1005C0000730FF007B08FE0C0318EA2AFF0BE32A22
:1005D000FB0100340310EF2AFE0C0318FB07FB0C91
:1005E000FD0CFF0BEC2AFB0CFD0C00349401930175
:1005F000093095008B138E018F018B17D613560887
:10060000FB007508F51BFF3CFE00FE13DF22FD0D0D
:100610007B0DF51FD607F51BD6025608760793000B
:0A06200003181414083095000800B8
:1007800002300F02031C0800EA1CDD2BA127F10830
:100790000319DD2B6E30D50071182D24F118322489
:1007A00071193724F1193C24E8006818F921E81878
:1007B00001226819FD21E81905220730EB050330F5
:1007C0008A006B088207E82B182C192C1A2C1B2C7A
:1007D000501C262C4008D500571A2D24D71A322435
:1007E000571B3724D71B3C24D6006108F50060084E
:1007F000F6005C1CF622C80B262C4C085C18053051
:10080000C8005C1CC00A5C1044084002031C262C73
:10081000C01B0E2C501E0E2CC001262C5012DC18B2
:1008200005125C1950105C1DC0035C1DC017262CFE
:10083000262C262C262C071C1F2C0710262CE908FA
:100840000319262C07140310E90C262CEB0A05309B
:100850006B020318EB018F01080005308A00D513E5
:100860005508820005308A00D517550882000630E9
:100870008A00D5135508820006308A00D51755081E
:020880008200F4
:100A000080340134033404340534063408340934A2
:100A10000A340B340D340E340F34113412341334C1
:100A2000143416341734183419341B341C341D3460
:100A30001E342034213422342434253426342734FF
:100A400029342A342B342C342E342F34303432349D
:100A50003334343435343734383439343A343C343C
:100A60003D343E34403441344234433445344634DA
:100A7000473448344A344B344C344D344F3450347A
:100A800051345334543455345634583459345A3418
:100A90005B345D345E345F346134623463346434B7
:100AA00066346734683469346B346C346D346E3456
:100AB00070347134723474347534763477347934F4
:100AC0007A347B347C347E34C4346434013401346D
:100AD0001134003401341134003400340034003453
:100AE0000034003400340034003400340034003466
:100AF0000034003400340034003400340034003456
:100B0000FF347E347C347B347A34793477347634F1
:100B1000753474347234713470346E346D346C34B2
:100B20006B346934683467346634643463346234F3
:100B300061345F345E345D345B345A345934583434
:100B40005634553454345334513450344F344D3476
:100B50004C344B344A3448344734463445344334B7
:100B6000423441343F343E343D343C343A343934F9
:100B700038343734353434343334323430342F3439
:100B80002E342C342B342A3429342734263425347B
:100B900024342234213420341E341D341C341B34BC
:100BA00019341834173416341434133412341134FD
:100BB0000F340E340D340B340A340934083406343F
:100BC0000534043403340134C4346434013401344E
:100BD0002234003401342234003400340034003430
:100BE0000034003400340034003400340034003465
:100BF0000034003400340034003400340034003455
:100C000080340034003401340234033404340634B4
:100C100008340A340C340E341134143417341A34B2
:100C20001D342134243428342C342F3433343734D5
:100C30003B343F34433447344B344F3452345634CE
:100C40005A345D346134643467346A346D347034DA
:100C500072347434763478347A347B347C347D3432
:100C60007E347E347E347E347E347D347C347B34FA
:100C70007A34783476347434723470346D346A343F
:100C80006734643461345D345A34563452344F34EA
:100C90004B34473443343F343B34373433342F34CC
:100CA0002C342834243421341D341A3417341434A9
:100CB00011340E340C340A3408340634043403344A
:100CC0000234013400340034C43464340134113447
:100CD00044340034013444340034003400340034EB
:100CE0000034003400340034003400340034003464
:100CF0000034003400340034003400340034003454
:100D000080340034003401340234033404340634B3
:100D100008340A340C340E341134143417341A34B1
:100D20001D342134243428342C342F3433343734D4
:100D30003B343F34433447344B344F3452345634CD
:100D40005A345D346134643467346A346D347034D9
:100D500072347434763478347A347B347C347D3431
:100D60007E347E347E347E347E347D347C347B34F9
:100D70007A34783476347434723470346D346A343E
:100D80006734643461345D345A34563452344F34E9
:100D90004B34473443343F343B34373433342F34CB
:100DA0002C342834243421341D341A3417341434A8
:100DB00011340E340C340A34083406340434033449
:100DC0000234013400340034C43464340134413416
:100DD0008834003401348834003400340034003462
:100DE0000034003400340034003400340034003463
:100DF0000034003400340034003400340034003453
:100E00003D1C08006C146D14EB011430B600071083
:100E10000130EB0507308A006B088207102F172F6F
:100E20006108F5006008F6000516D6011A2F7F301C
:100E3000D6001A2F701A432F6B18232F7019F60A39
:100E40007018F603272F7019F50A7018F503503043
:100E50007018EC007019ED00C8307602C830031825
:100E6000F600503076025030031CF600F51F3E2F7E
:100E7000A0307502A030031CF500432F64307502CA
:100E800064300318F5007F30D6006B1CD601F622C3
:100E9000EA017927701C4E2F6D1B7016701D522FA2
:100EA0006C1B7016701E572FEB0A6B1C682F0710F7
:100EB000B60B5F2F07143C306B180A30B600640085
:100EC0000A300F02031C5F2F8F01701A082F1A2F90
:100ED0007508E1007608E000603084000408BC007A
:100EE0000008BB00B021840A68300402031C6E2F86
:100EF0000800F0010A30851DEC078519EC027830F6
:100F00006C020319701479300318EC0015306C0270
:100F10000319F0141430031CEC000A30051CED0713
:100F20000518ED0278306D02031970157930031839
:100F3000ED0015306D020319F0151430031CED009F
:100F40000800F1010A30871DEE0702308719EE0212
:100F500078306E020319711479300318EE001530E1
:100F60006E020319F1141430031CEE000A30071E40
:100F7000EF070230071AEF0278306F02031971157C
:100F800079300318EF0015306F020319F115143092
:060F9000031CEF00080045
:084000000C00000004000500A3
:02400E00CC33B1
:1042000001008100820084008800B100B200B40087
:10421000B800A100A200FF00FF00FF00FF00FF00A8
:104220000000010001000100010001000100010087
:10423000010001000100FF00FF00FF00FF00FF0080
:10424000010000000000000000000000000000006D
:10425000000000000000FF00FF00FF00FF00FF0063
:10426000FF00FF00FF00FF00FF00FF00FF00FF0056
:10427000FF00FF00FF00FF00FF00FF00FF00FF0046
:10428000FF00FF00FF00FF00FF00FF00FF00FF0036
:10429000FF00FF00FF00FF00FF00FF00FF00FF0026
:1042A000FF00FF00FF00FF00FF00FF00FF00FF0016
:1042B000FF00FF00FF00FF00FF00FF00FF00FF0006
:1042C0007D00FC007D00FC007D00FC007D00FC000A
:1042D000FF00FF00FF00FF00FF00FF00FF00FF00E6
:1042E0000000000000000000FF00FF00FF00FF00D2
:1042F000FF00FF00FF00FF00FF00FF00FF00DD00E8
:00000001FF
